:020000020000FC
:10000000A2C018C017C016C015C014C013C012C0BB
:1000100011C010C00FC00EC00DC00CC00BC00AC074
:1000200009C008C007C006C005C004C003C002C0A4
:1000300001C000C05F9AEF93FF93E8EEF3E0EF9307
:10004000FF93ECECF7E03197F1F7FF91EF913197E7
:1000500011F000C0F4CFEF91FF91439AEF93FF931B
:10006000E8EEF3E0EF93FF93ECECF7E03197F1F774
:10007000FF91EF91319711F000C0F4CFEF91FF9114
:100080004398EF93FF93E8EEF3E0EF93FF93ECECEC
:10009000F7E03197F1F7FF91EF91319711F000C040
:1000A000F4CFEF91FF915F9808952A985C98299A70
:1000B00008952A985C9A299808952A9A5C98299814
:1000C0000895E3E0E093B000E3E2E4BD0895E3E0E7
:1000D000E4BDE3E2E093B0000895E3E0E4BDE3E8CB
:1000E000E093B0000895303059F0313069F032308B
:1000F00071F0333079F0343081F0DBDF33270FC01B
:10010000D8DFEBDF31E00BC0D0DF32E008C0DFDF4B
:1001100033E005C0D2DF34E002C0D3DF35E008951C
:10012000EF93FF93E8EEF3E0EF93FF93ECECF7E04F
:100130003197F1F7FF91EF91319711F000C0F4CFB3
:10014000EF91FF910895E3E0EEBFE0E0EDBFF8949A
:10015000E0E1E5BF239A539A559A229A549A219A3C
:10016000579A3B9AEE27E5B9E8B9EBB928E7E22FB1
:10017000E8BDE093B300E093B400E3E0E4BDE1E068
:10018000E5BDE3E0E093B000E1E0E093B100E2E040
:10019000E6BD50DFEF93FF93E8EEF3E0EF93FF93BC
:1001A000ECECF7E03197F1F7FF91EF91319711F017
:1001B00000C0F4CFEF91FF9133275F9A439A93DF0A
:1001C000AFDF5F9843988FDFABDF5F9A439A8BDF97
:1001D000A7DF5F98439887DFA3DF5F9A439A83DFA7
:1001E0009FDF5F9843987FDF9BDF5F9A439AE5CF5D
:00000001FF
